:10000000BDC20000F3C20000F1C20000EFC2000058
:10001000EDC20000EBC20000E9C20000E7C2000030
:10002000E5C20000E3C200000C94B72C0C949F2D95
:100030000C946C2CDBC20000D9C20000D7C20000B7
:10004000D5C20000D3C20000D1C20000CFC2000060
:10005000CDC200000C94932CC9C20000C7C200009E
:10006000C5C20000C3C20000C1C20000BFC2000080
:10007000BDC20000BBC20000B9C20000B7C2000090
:10008000B5C20000B3C20000B1C20000AFC20000A0
:10009000ADC20000ABC20000A9C20000A7C20000B0
:1000A000A5C20000A3C20000A1C200000501090210
:1000B000A10185020901A1000509190129081500FE
:1000C0002501950875018102050109300931158165
:1000D000257F95027508810609381581257F9501D0
:1000E00075088106050C0A38021581257F95017572
:1000F000088106C0C005010980A101850319012AF4
:10010000B700150126B700950175108100C0050CD8
:100110000901A101850419012AA002150126A002E6
:10012000950175108100C005010906A1018506052C
:100130000719E029E71500250195087501810205D9
:1001400007190029EF1500250195F07501810205B9
:10015000081901290595057501910295017503910D
:1001600001C00660FF0961A1010962150026FF00B8
:100170009520750881020963150026FF00952075FA
:10018000089102C005010906A101050719E029E748
:1001900015002501950875018102950175088101F9
:1001A0000507190029FF150026FF0095067508812F
:1001B000000508190129051500250195057501910E
:1001C00002950175039101C00000000000000000CD
:1001D000000000000000000000000000000000001F
:1001E0000000000000000000000000007E0F00D4AE
:1001F000FFFFFFC7000000780000000000000000C3
:100200002A2B280000000000000000000000000071
:1002100000000029000000002C1E3420212224347C
:100220002627252E362D3738271E1F20212223244E
:1002300025263333362E37381F0405060708090AEA
:100240000B0C0D0E0F101112131415161718191A86
:100250001B1C1D2F3130232D350405060708090A04
:100260000B0C0D0E0F101112131415161718191A66
:100270001B1C1D2F3130354C09025B00030100A00F
:10028000FA09040000010301010009211101000124
:10029000224400070581030800010904010002034C
:1002A000000000092111010001222200070582033C
:1002B00020000107050303200001090402000103D7
:1002C00000000009211101000122B6000705840386
:1002D0002000011201000200000008434C2004002D
:1002E00001010203011C037600690061006C003A01
:1002F00000660036003400630032006200330063A1
:100300000000000C037300770069007300730000A5
:1003100000100342007200650067006F006C006906
:100320000000000403090429001E001F0020002112
:10033000002200230024002500260027002D002E87
:100340000031004C002B0014001A000800150017A3
:10035000001C0018000C00120013002F0030002AAF
:10036000000000E00004001600070009000A000B6E
:10037000000D000E000F00330034002800000000C4
:1003800000E1001D001B000600190005001100100F
:1003900000360037003800E500215200000000E37D
:1003A00000E2000000000000002C0000000000003F
:1003B000000000E6000000E4000000000035003A04
:1003C000003B003C003D003E003F00400041004239
:1003D0000043004400450049004C00390001000181
:1003E0000001000100010001000100460077004803
:1003F0000052000100010000000100AA00A900A8AD
:1004000000B0000100550054004A004B0050004F5E
:1004100000010000000000010001000100010001D6
:10042000000100570056004D004E00510001000130
:1004300000000000000100010000000000000001B9
:1004400000000000000000000001000000010000AA
:10045000000000FD377A585A000004E6D6B4460280
:1004600000210116000000742FE5A3E002D000E88F
:100470005D003D8889A654750A36E182AEFA7A1A83
:10048000A6FCA2ED4954B48A5E7177BBD0558EFFAD
:100490000917CD130C292F7E08A206F4B9E5A0FE9A
:1004A000A15BBEAFBDEA7B1A2C60BA3FAEE9A19B4F
:1004B000293FF6D9F65FB7C703CAA4B7C5D24C9E89
:1004C0009C12A9CC4D80EEA98D22DE0E4027116131
:1004D00018DF499B636B0C9FFF007F86D7F9853B34
:1004E000A8F8F722A34E4BC272CCDC4AB0607D81E3
:1004F0006383FBB9128F689301C7F1B22384877EAF
:10050000DEEEE01576AD15E379EF9304D10CD5C29C
:10051000E73F55598FCDF80F5780094642A4A9A748
:10052000800829AB596A711FA9AB49E4D1E8656A13
:10053000D2E1EF761530AEE19DA13A2C8707ADE20E
:10054000D356028935D24DEA00114080E1D9DB75DE
:100550003F53CE30C3F42EEC6B00006E071E4010EC
:1005600016677600018402D105000064CD97A4B11E
:10057000C467FB020000000004595A0011241FBE8A
:10058000CFEFDAE0DEBFCDBF04B603FE18C0809126
:10059000030590910405A0910505B09106058730EB
:1005A000904BA740B04B59F41092030510920405EC
:1005B0001092050510920605E0E0F8E3099511E0B8
:1005C000A0E0B1E0EEE9FEE502C005900D92AA3A86
:1005D000B107D9F725E0AAEAB1E001C01D92A33026
:1005E000B207E1F70E947A250C94D32E09CD9C0125
:1005F0009A9581159F4118F5F32FF270EE27832FFE
:100600008170732F74706627532F5870442734FFFE
:100610000CC08295807FEF2B09F08062672B09F078
:100620008064452B69F080680895EF2B09F08260A3
:10063000672B09F08460452B19F08860089580E0ED
:100640000895CF93DF93EB01D2DFFE010995DF918F
:10065000CF910895982F92959F7024E0911102C038
:1006600020E0982F892F86958695811511F02E5FB1
:10067000982F892F8695820F08958093FF040895FF
:1006800080930005089521E030E001C0220F8A9593
:10069000EAF780910005822BF3CF21E030E0A90139
:1006A00002C0440F551F8A95E2F7CA0180959091C8
:1006B00000058923E5CF292F953090F58F3080F5FF
:1006C00090E03FE0239F800D911D1124282F27707B
:1006D00041E001C0440F2A95EAF723E096958795FB
:1006E0002A95E1F7FC01EE0FFF1FE80FF91FEA5F03
:1006F000FC4F20E030E070E05191DF01CB01022E91
:1007000002C0969587950A94E2F7817081958527B6
:10071000842385278E932F5F3F4F2330310561F768
:100720000895292F953078F58F3068F590E03FE0F7
:10073000239F800D911D1124682F677023E09695EB
:1007400087952A95E1F7FC01EE0FFF1FE80FF91FCF
:10075000EA5FFC4F40E050E080E0219130E0062E5F
:1007600002C0369527950A94E2F721703327042EAC
:1007700001C0220F0A94EAF7822B4F5F5F4F43308C
:10078000510559F7089580E008959091000521E002
:1007900030E0F90101C0EE0F8A95EAF7D90102C0F5
:1007A000AA0FBB1F6A95E2F7EA2B01C0220F4A95F8
:1007B000EAF7892F8E23E81303C0892F822B60CF9D
:1007C0002095822F8923FBCF8091B4029091B302B0
:1007D000981301C008958F5F8770FACF90914B04F2
:1007E0008095892380934B04282F2770211110C0F6
:1007F000891771F09091020592FF0AC0869586953F
:1008000086954BDF10924B0410924D0410924C04CD
:10081000089590914804982B909348040895982F38
:10082000909580914804892380934804089580918D
:100830004704811531F01092470410924F04109232
:100840004E040895803E9105D9F1C8F48133910595
:1008500009F482C048F48932910509F472C08A32E1
:10086000910509F480C0089589339105E9F0823833
:100870009105D1F08533910509F45EC00895843E59
:100880009105D9F148F4823E910539F1833E9105F5
:1008900049F181EE90E00895863E9105C9F1873EC9
:1008A000910509F43EC0089520910105237021119E
:1008B00064C02091020523FF14C089E290E00895EE
:1008C0002091010520FD45C03091020530FF09C08F
:1008D00024FD24C083EE90E008952091010522FDBF
:1008E000F7CF08952091010522FD44C03091020503
:1008F00030FD43C024FFF5CF11C02091020521FF38
:10090000F0CF8091010584FD09C087EE90E0089545
:100910002091010523FFE5CF24FFF7CF80E090E091
:1009200008952091010523FD2BC03091020531FF70
:10093000E1CF84EE90E008952091010525FFD1CF0D
:10094000BCCF2091010525FD1EC02091020523FF8B
:10095000C8CF89E390E008952091010526FFC1CF1B
:100960008AE290E008952091010526FFBACF81E345
:1009700090E0089582EE90E0089580EE90E0089572
:1009800086EE90E0089585E390E00895909101054A
:1009900092FF10C041E0282F2471243009F040E07C
:1009A00031E0282F2871283009F030E0431711F08A
:1009B0002CE0822793FF10C041E0282F24712431BE
:1009C00009F040E031E0282F2871283109F030E0AB
:1009D000431711F02CE082273091020530FF10C040
:1009E00051E0282F2171213009F050E041E0282FFB
:1009F0002871283009F040E0541711F029E08227CF
:100A000031FF10C041E0282F2171213109F040E071
:100A100031E0282F2871283109F030E0431711F018
:100A200029E0822794FD877E08951F93CF93DF935B
:100A300009DFEC01811522E5920708F052C081150B
:100A400040E5940708F0CDC0803E910520F58D3C2F
:100A5000910508F0A1C0883A910570F4853A910596
:100A600008F097C081309105B9F10497813A91055A
:100A700098F1C0E0D0E030C0885A91094B97C8F790
:100A8000C85AD0E0CC0FDD1FC25CDE4F0990D88180
:100A9000C02DD46421C0811550E49507B0F4C11570
:100AA00080E2D80708F0B3C0C83ED105A8F0CE0157
:100AB0009A9581159F41E8F68D2F68DF182FCE019A
:100AC0009927C0DEEC01D12B07C09927BBDECC27CC
:100AD000DF70C82BD92BD06ACE01DF91CF911F9147
:100AE0000895803842E59407C8F5803652E59507A9
:100AF00008F05BC0C03482E5D807D0F4C03292E57C
:100B0000D90708F04BC08C2F8695869520E2829FEE
:100B1000C0011124C37021E030E0A90102C0440FDC
:100B2000551FCA95E2F7EA01C82BD92BDD68D4CF4F
:100B30008C2F86958695877050E2859FC001112481
:100B4000C37021E030E0A90102C0440F551FCA95CF
:100B5000E2F7EA01C82BD92BDC68BECF803C52E516
:100B6000950758F48F71C03AD245A0F590E0982FC0
:100B70008827EC01C46FD06AAFCF805C9245809724
:100B800008F077CFDC2FCC27CC27DF71C06FD06A7D
:100B9000A3CFA497D064A0CFD0659ECFCF71D0E073
:100BA000DC2FCC27C16FD06A97CF8695869587704A
:100BB00020E2829FC0011124C37021E030E0A9012E
:100BC00002C0440F551FCA95E2F7EA01C82BD92B82
:100BD000DA6882CFDBDEC82FD0E0DC2FCC27D062F2
:100BE0007BCF8F71D3DE93E0CC0FDD1F9A95E1F7B9
:100BF000CC27DF70282F30E084FF05C050E1859FAF
:100C0000900111243327C22BD32BD06965CF8D2FB0
:100C10008F71BCDE182FCE01992714DEEC01D12B89
:100C2000DECF80E00895F894E82FE295EF70F0E0D1
:100C300041A18F7021E030E0B90102C0660F771F3B
:100C40008A95E2F7CB01962F9095942391A392A1D8
:100C5000892B82A37894089581152CE7920741F49B
:100C60002091800230918102232B11F480E090E0EA
:100C70000895E0ECF3E080E090E068EE73E24BE092
:100C800054E22DE734E277836683518740873387C8
:100C9000228797878687019670968830910599F705
:100CA00008951092910410929004E0E5F4E085819B
:100CB000811102C014821682379684E0E838F80762
:100CC000B1F70895AC013091930460919204232F01
:100CD000621301C00895822F90E0FC01EE0FFF1F08
:100CE000E857FB4F0190F081E02DE417F50791F4F0
:100CF00067E0649FF001659FF00D1124E05BFB4FFE
:100D000041E044832313E6CF0196837099278093B3
:100D1000930408950196282F2370DACFFC01848173
:100D2000862381110AC082818115B9F068239085DC
:100D300093FF05C081E061110FC080E00895282F66
:100D400022952F708F70282B962F92959F706F7021
:100D5000962B81E02913F1CF089581E008950F9338
:100D60001F93CF9301E010E0082E01C0000F0A94FA
:100D7000EAF7C09146049C2F9023911115C09091E1
:100D80004B04969596959695891306C010924B0440
:100D900010924D0410924C0476DCC027C093460498
:100DA000CF911F910F91089578DCF7CF282F35EB65
:100DB0002303C001112497FF04C080589109892F93
:100DC000089580589F4FFBCF8091260380FD14C06B
:100DD00081FD14C082FD16C080912503811581F02C
:100DE0008E3180F420E5829FC00111246EE170E015
:100DF0000E94EA2D862F089584E1089588E20895DF
:100E000088E0089580E508958091260380FD17C04D
:100E100081FD17C082FD19C080912403811599F0CE
:100E2000883298F428E0829FC001112468E270E0C3
:100E30000E94EA2D6115710551F0862F089562E038
:100E4000FCCF64E0FACF61E0F8CF68E0F6CF81E054
:100E50000895FA01309709F009950895E091A902E3
:100E6000F091AA02309739F00190F081E02D30978F
:100E700011F00995089580E00895A3E0B0E0E3E45F
:100E8000F7E00C941A2E9C018091F2019091F301ED
:100E900082179307B1F03093F3012093F201E091B0
:100EA000A902F091AA02309761F00084F185E02D4B
:100EB000309739F083E089833B832A83CE01019602
:100EC00009952396E2E00C94362EA3E0B0E0EBE621
:100ED000F7E00C941A2E9C018091F0019091F101A1
:100EE00082179307B1F03093F1012093F001E09164
:100EF000A902F091AA02309761F00084F185E02DFB
:100F0000309739F084E089833B832A83CE010196B0
:100F100009952396E2E00C94362E90910E019130C3
:100F200091F0AEEAB1E0EFEF90E02D91821751F031
:100F3000EF3F19F4211101C0E92F9F5F9630A9F707
:100F4000EF3FC9F408959091010597FFEACFE82F8C
:100F5000E695E695E695803FA8F7F0E0EC54FE4F65
:100F6000877021E030E001C0220F8A95EAF7828184
:100F7000822B828308950E2E000CFF0BE455FE4F4A
:100F8000F8CF90910E01913021F49091010597FDD9
:100F90000CC0EEEAF1E09191891302C0DF011E92CC
:100FA00051E0E43BF507B9F70895E82FE695E6959B
:100FB000E695803FC8F7F0E0EC54FE4F877021E0E3
:100FC00030E0A90102C0440F551F8A95E2F7CA011B
:100FD0008095928189238283089580910D010895DF
:100FE0002FB7F8948091EC019091ED01A091EE0162
:100FF000B091EF012FBF0895CF93DF93C0914804C4
:1010000080914A04C82B809147048115F1F0E8DFF4
:1010100020914E0430914F04821B930B88389341EA
:1010200008F005DCD091470480910E01813021F455
:101030008091010587FD13C086E02EEA31E090E043
:10104000815088F49111F3DBCD2B80913C03809586
:101050008C2390913B03892BDF91CF9108958EE1F2
:1010600026EB31E0ECCFF90141919F01411541F3AD
:101070009F5FE6CF962F2091020522FF0EC0682FBA
:10108000660F660F660F692B60934B04FCDAA8DFCE
:1010900090934D0480934C040895F5CA90914704B1
:1010A000292F2823211559F08095892380934704FF
:1010B000811531F095DF80934E0490934F0408958D
:1010C00080E090E0F8CF8CDF2091290330912A0353
:1010D000232B211521F080936F02909370022091B1
:1010E0002B0330912C03232B211521F080936D02CB
:1010F00090936E02E091A902F091AA02309759F004
:101100000680F781E02D309731F082E0809327034D
:1011100087E293E009950895611509F441C0E3E37E
:10112000E80FE33148F4F0E0EB52F14D0C94FD2D63
:101130004BDE819580932A03C6CF46DEFBCF44DE8B
:10114000819580932903F8CF3FDEFBCF5DDE80934E
:101150002B03F2CF59DE8195FACF56DE819580932D
:101160002C03EACF51DEFBCF815D990B21E030E00B
:1011700001C0220F8A95EAF780912803822B809381
:101180002803DACF80912603816080932603D4CF91
:10119000809126038260F9CF809126038460F5CF89
:1011A000409129038D3C59F480912A0387FF0DC09B
:1011B00010922A03411559F41092250308C08E3C61
:1011C00081F480912A0318169CF3411581F08091D7
:1011D0002B0390912C03892B8111AECF1092240305
:1011E000ABCF8F3C41F447FFF0CF109229038091A1
:1011F0002A038115E0CF803D19F41416B4F3E5CF2E
:1012000090912B03893D29F41916FCF610922B03BB
:10121000DCCF8A3D19F497FFD8CFF8CF90912C03FB
:101220008B3D29F497FFD1CF10922C03CECF8C3D6C
:1012300019F41916CCF3C9CF9FE2980F983090F4A7
:10124000815D990B21E030E0B90102C0660F771F84
:101250008A95E2F7CB0180959091280389238093AA
:101260002803B3CF8D3D31F4809126038E7F809388
:101270002603ABCF8E3D21F4809126038D7FF7CFDF
:101280008F3D09F0A2CF809126038B7FF0CF2FB73F
:10129000F8946091EC017091ED018091EE019091D4
:1012A000EF012FBF0895CF92DF92EF92FF92CF937D
:1012B000DF93D82FC92FC090BA03D090BB03E09022
:1012C000BC03F090BD03E3DF6C197D098E099F0913
:1012D000643F71408105910510F1D9DF6B017C01FC
:1012E00082E390E0A0E0B0E0C0926902D0926A028E
:1012F000E0926B02F0926C0280936502909366021A
:10130000A0936702B0936802D093B803C093B90367
:10131000DF91CF91FF90EF90DF90CF90089584EF11
:1013200091E0A0E0B0E0E0CFFC019B018091E20100
:101330009091E3018617970740F0672B29F480917D
:10134000E8008E778093E800C90140E0009741F4FF
:10135000411106C08091E80082FF2FC080E008950F
:10136000209182022115A9F12530A9F12091E800F0
:1013700023FD2DC02091E80022FDECCF2091E80054
:1013800020FFE4CF3091F3002091F200009719F094
:101390002830310558F041E02830310509F040E0AF
:1013A0002091E8002E772093E800D0CF4191409320
:1013B000F10001972F5F3F4FE9CF809182028115A5
:1013C00041F0853041F08091E80083FFC3CF81E098
:1013D000089582E0089583E008958091DC0187FFFD
:1013E00013C08091E80082FF06C08091E8008B77EF
:1013F0008093E8000895809182028111F2CF0895D0
:10140000809182028115D9F38091E80080FFF8CFA6
:101410008091E8008E77ECCF2091E4003091E500D8
:1014200095E6A9012091EC00822F817020FF06C073
:101430008091E80080FF06C080E008952091E800D8
:1014400022FD1AC080918202811589F0853089F0D1
:101450008091EB0085FD0FC02091E4003091E50004
:1014600042175307F9F29A95E1F684E0089582E075
:10147000089583E0089581E00895E8EDF0E080812B
:101480008E7F80831092E2001092DA001092E100C9
:10149000A0EEB0E08C9181608C9380818F77808307
:1014A00019BCA7EDB0E08C918E7F8C9380818F7EEC
:1014B00080831092DB010895E091A902F091AA02C5
:1014C000309739F00284F385E02D309711F060E217
:1014D00009950895982F9093E900891771F07091FC
:1014E000EC002091ED005091F00021FD09C09F5FBC
:1014F000973089F78093E9000895762F242F50E0E4
:101500003091EB003E7F3093EB003091ED003D7F5A
:101510003093ED003091EB0031603093EB0070932D
:10152000EC002093ED005093F0002091EE0027FD99
:10153000DECF0895A0E0B0E0E0EAFAE00C94142ECB
:10154000C8EDD0E088818F7E8883E7EDF0E0808170
:101550008160808384E082BF81E08093DB018881A9
:101560008E7F888302EE10E0F80110821092DA007C
:1015700081EEC82ED12CF601108288818F77888366
:1015800088818068888388818F7D888319BC1092C8
:1015900082021092DA01109259021092D90190EE53
:1015A000E92EF12CF70180818B7F80838881816017
:1015B000888342E060E080E08DDFF60180818E7FED
:1015C0008083F8018081816080838081886080834E
:1015D000F70180818E7F8083888180618883CDB789
:1015E000DEB7E8E00C94302EE091B4029091B302A3
:1015F00029E0E91302C080E00895AE2FB0E02E9FED
:10160000F0011124EB54FD4F3181361306C03081B7
:10161000381303C03581341304C0FD013196E770DF
:10162000E8CF81E0089581E08093E00080E280933C
:10163000D8001092C9008FE19EE40197F1F700C035
:10164000000087E090EBDC01809303059093040594
:10165000A0930505B093060588E19CE00FB6F894C9
:10166000A895809360000FBE90936000FFCF0F930A
:101670001F93CF93DF938B01EA0190918202943004
:1016800051F58093E9008FEF9091E80095FD06C039
:1016900095ED9A95F1F700008A95B1F78091E800F1
:1016A00085FF19C0B9DE811111C08091E80085FD68
:1016B00006C08091E8008E778093E800F3CFF801B0
:1016C00081918F018093F100219779F78091E80053
:1016D0008E778093E800DF91CF911F910F9108954D
:1016E000792F603229F440E250E0682F82E0BFCFCA
:1016F0000895CF93DF93D82FC92F48E050E0682F8B
:10170000792F81E0B4DF88E0ED2FFC2FA4EEB1E06B
:1017100001900D928A95E1F7DF91CF910895BC0178
:1017200040E250E084E0A3CFBC0146E050E084E01A
:101730009ECFBC0143E050E084E099CF9091020538
:1017400092FB222720F9281771F080FB92F99093E1
:101750000205609101057091020584E090E00E940D
:10176000B82E82E03BC808951F93CF93DF93962F46
:10177000122F632F8430D8F49530C8F44F30B8F46A
:10178000C42FD0E0CC0FDD1F2EE1929FC00DD11DE4
:10179000112496E9899FC00DD11D1124CE0189968F
:1017A0000E949E2E612FCE018A960E949E2EDF916E
:1017B000CF911F91089580910E01813061F5809144
:1017C000010587FF28C018DC8093B50140E250E096
:1017D00069E872E084EB91E00E945E2E892BD1F0E3
:1017E00080E2E4EBF1E0A9E8B2E001900D928A9585
:1017F000E1F7E091A902F091AA02309759F0048034
:10180000F581E02D309731F086E08093B40184EBD0
:1018100091E009950895F0DB8093AC0148E050E039
:101820006BEA72E08CEA91E00E945E2E892B91F3C4
:1018300088E0ECEAF1E0ABEAB2E001900D928A9523
:10184000E1F7E091A902F091AA02309719F3028022
:10185000F381E02D3097F1F28CEA91E0DACF811537
:1018600019F00E940904A7CF0895811531F09091D5
:101870004A04892B80934A049ECF0895CF93C82FA2
:101880008115C1F08CEF8C0F813A80F580910E01AB
:10189000813021F48091010587FD0EC0EEEAF1E070
:1018A0008191C817F9F021E0E43BF207C9F78C2FCA
:1018B00034DB81DFCF910895EC2FE695E695E69530
:1018C000F0E0EC54FE4F828190E04C2F477021E015
:1018D00030E002C0220F331F4A95E2F782239323A0
:1018E000892B29F38C2F4DDB66DFE1CF80E28C0F53
:1018F000883048F4C77081E001C0880FCA95EAF7C4
:101900000E940904D6CF8BE58C0F833030F42C2F46
:101910002452330BC901B1DACDCFE8E5EC0FEB313E
:1019200048F4F0E0EE0FFF1FEC58FE4F80819181EC
:10193000CCDAC0CF83E38C0F833108F0BBCF61E0FA
:101940008C2FEADBB7CFCF93DF93EC01805E910958
:10195000089720F065E37CE0209711F46FE27CE0CB
:10196000CE010E9421038C2F89DFDF91CF91089552
:10197000811541F19CEF980F913A10F402DB1BCFD7
:1019800090E2980F983050F4877091E001C0990F61
:101990008A95EAF7892F0E940F04F1CF9BE5980FF3
:1019A000933018F480E090E068CA98E5980F9B3176
:1019B00018F480E090E089CA93E3980F933110F413
:1019C00060E0AACB08951F93CF93DF93182FEB010C
:1019D00055DF209731F4812FCBDFDF91CF911F911D
:1019E00008958FE99FE00197F1F700C0000021976B
:1019F000F0CF811519F00E940F04DDCE08958115F6
:101A000039F0809590914A04892380934A04D3CE7B
:101A1000089580913703811521F082E2F0DF109262
:101A2000370308951092480480910E01813011F51A
:101A30008091010587FF1EC0E6EBF1E08EE1DF013A
:101A40001D928A95E9F780E090E017DA80E090E057
:101A50003CDA10924A04AFDE86E0E7E2F3E0DF0111
:101A60001D928A95E9F71092250310922403109293
:101A7000260329CBEEEAF1E086E0E1CFD3DF2FEFBA
:101A800084E39CE0215080409040E1F700C00000DA
:101A900088E19CE00FB6F894A895809360000FBE93
:101AA00090936000FFCFAAE2B0E0E9E5FDE00C947E
:101AB000192E8CED91E0FC0101962091F10020831C
:101AC00021E0843E9207B9F78091DD01893009F465
:101AD00057C0C8F4823009F4B2C0833009F482C020
:101AE000813081F18091E80083FFE6C08091DC01C4
:101AF0009091DD019A3008F0DFC0E92FF0E0E85165
:101B0000F14D0C94FD2D8A3009F489C08B3051F7CA
:101B10008091DC01813231F78091E0019091E10107
:101B2000892B01F78091E800877F8093E80055DCDE
:101B300081E09091DE01911101C080E080930E015F
:101B400071DFD0CF8091DC01813A61F68091E800AD
:101B5000877F8093E8008091E0019091E101892BDB
:101B600059F060E080E090E070E0DEDB8091E8001A
:101B70008B778093E800B6CF68E084EE91E0F4CFF5
:101B80008091DC01813209F0ADCF8091E00190912C
:101B9000E1018D7F892B09F0A5CF8091E800877F37
:101BA0008093E8008091E80082FF17C09091F300D5
:101BB0008091F200029731F48091F100813011F0B0
:101BC000863021F48091F10080930D018091E8002E
:101BD0008B778093E80001DC85CF809182028111B0
:101BE000E1CF80CF8091DC01813A09F07BCF8091F9
:101BF000E0019091E101892B09F074CF8091E80018
:101C0000877F8093E8008091E80080FFFCCF80917F
:101C10000E018093F1008091E8008E77DACF8091F9
:101C2000DC01813209F05ECF8091E800877F8093EC
:101C3000E800D3DB8091DF0180930C0153CF8091CA
:101C4000DC01813A09F04ECF8091E800877F8093D4
:101C5000E8008091E80080FFFCCF80910C01D9CF93
:101C6000803889F0823841F58091E0018F708730AB
:101C700018F58093E9008091EB0085FB882780F9B7
:101C80001092E90006C080915902880F9091D90105
:101C9000892B9091E800977F9093E8008093F10062
:101CA0001092F1008091E8008E7723C0811116C058
:101CB0008091DE01813009F18091E80083FF0AC044
:101CC0008091E800877F8093E8008091EB0080623C
:101CD0008093EB00AA96E3E00C94352E823061F7F6
:101CE0008091DE01811581F01092E9008091E80079
:101CF000877F8093E80071DBDFCF81E0933009F0CC
:101D000080E080935902F0CF8091E0018F702FEF37
:101D1000280F263088F68093E9002091EB0020FF01
:101D2000E3CF933031F48091EB0080628093EB003D
:101D3000DBCF9091EB0090619093EB0021E030E0DD
:101D4000A90102C0440F551F8A95E2F74093EA00AB
:101D50001092EA008091EB008860E8CF8111ACCF4F
:101D60001091DE011F778091E3008078812B8093B2
:101D7000E3008091E800877F8093E8002EDB80916C
:101D8000E80080FFFCCF8091E30080688093E3004F
:101D900083E0111101C082E0809382028DCF8058D0
:101DA000823008F089CF8091DE019091DF018C3D77
:101DB00053E0950791F583E08A838AE289834FB7E0
:101DC000F894DE01139620E03EE051E2E32FF0E0CC
:101DD00050935700849120FF03C082958F703F5F1E
:101DE0008F708A30C0F0895C90E08D939D932F5F57
:101DF000243161F74FBF8091E800877F8093E8002E
:101E00006AE270E0CE0101968FDA8091E8008B776C
:101E10008093E80051CF805DE7CF292F332723300F
:101E2000310509F44EC078F52130310509F488C038
:101E30008BE590E0E8E7F2E02230310509F03CCF95
:101E40002091E800277F2093E8002091E201309163
:101E5000E3018217930708F49C0140E02115310546
:101E600009F073C0411171C08091E80082FDCDCFAF
:101E700080918202811549F2853039F28091E80023
:101E800083FFF2CFC2CF8091E0019091E101213236
:101E9000310509F446C02232310509F00DCF8330F7
:101EA000910508F009CFFC01EE0FFF1FE25EFE4F27
:101EB0000190F081E02D855E9E4FDC018C9190E0D9
:101EC00010C09C013327823021F12330310568F4A2
:101ED000232BB9F4E3E2F3E0E4918E2F90E0E3E208
:101EE000F3E0009709F4E8CEABCF2330310509F0D9
:101EF000E3CEE5EEF2E0E4918E2F90E0E5EEF2E045
:101F0000F0CFE1E1F3E0E4918E2F90E0E1E1F3E046
:101F1000E8CFE3E0F3E0E4918E2F90E0E3E0F3E03C
:101F2000E0CF8330910508F0C7CEFC01EE0FFF1F14
:101F3000EC5DFE4F0190F081E02D89E090E080CFD4
:101F400082E190E0E3EDF2E07BCF809182028115A7
:101F500009F45BCF853009F458CF8091E80083FD08
:101F600054CF8091E80082FD7FCF8091E80080FF10
:101F700075CF9091F3008091F2002115310519F091
:101F80008830910550F041E0089709F040E08091D9
:101F9000E8008E778093E80061CF44914093F10090
:101FA0003196215031090196E8CF803809F084CE6E
:101FB0008091E800877F8093E8008091DA01809328
:101FC000F10070CE811178CE1091DE01123008F050
:101FD00073CE8091E800877F8093E8001093DA0148
:101FE000FCD91115D9F084E08093820242E061ECC3
:101FF00081E070DA42E261EC84E06CDA42E261ECAA
:1020000082E068DA42E260EC83E064DA8091820286
:10201000843051F482E080930F014ECE8091E30032
:1020200087FDE1CF81E0E0CF81E0F5CFCF93DF9373
:10203000EC014A855B856E857F850E9429079B811F
:10204000909580914A04892380934A048C810E9450
:102050000F04B1DB86E0FE0111928A95E9F7DF916A
:10206000CF910895CF93DF93EC018D8181FD13C053
:1020700082608D8380914A049B81892B80934A04DE
:102080008C810E94090497DB488559856E857F8580
:10209000CE010E94290710924104109240048D81C4
:1020A00080FD02C0CE01C2DFDF91CF9108951F9362
:1020B000CF93DF93182FA091B603B091B703109779
:1020C00009F448C01092B9031092B80310923C036F
:1020D00010923B031696CD91DC911797CE019A95FD
:1020E00081159F4108F4D07ED1E0C11101C0D0E03C
:1020F0001996ED91FC911A97309731F01B966D91DE
:102100007C9180E00995D823D11539F08CEF8C0FA4
:10211000813A20F58C2F0E94C1071115A1F0E091A2
:10212000B603F091B703808584FD0DC08091B5039F
:10213000811549F0808191819C01215031092F3313
:102140003E4708F4B0D837DB1092B7031092B603BD
:102150001092B503DF91CF911F9108952CDB8C2F46
:1021600007DCDBCF0F931F93CF93DF93843030F5E1
:10217000653020F54F3010F5C42FD0E0CC0FDD1FB7
:102180002EE1629FC00DD11D112436E9839FC00D41
:10219000D11D1124CE0189960E94822E082F10E0B5
:1021A000102F0027CE018A960E94822E9801282B9C
:1021B000C901DF91CF911F910F91089580E090E0C8
:1021C000F8CF462F672F2091850230918602232B6E
:1021D00081F4703F39F4403F61F480918302909123
:1021E00084020895753028F44F3018F4843008F4D0
:1021F000B9CF80E090E00895A0E0B0E0E2E0F1E146
:102200000C94152E7C01009100058091FF04082B91
:10221000C3E0D0E010E0C8010C2E02C09595879570
:102220000A94E2F780FD09C02197A8F7D12C8D2DE3
:10223000CDB7DEB7E7E00C94312EDC2EB7018C2F42
:10224000C0DF0E941505019779F3F1CF0F931F931B
:10225000CF93FC0187819085009789F48581008167
:102260001181811581F0611571F0C801C5DFC82F9A
:10227000682FC8010E945B03B8018C2FA2DFCF91A9
:102280001F910F910895C8010E949103C82FF4CFA8
:10229000CF93DF93D82FC92FAFDF6D2F7C2F91DF26
:1022A0000E941505DF91CF910895FC01848181156D
:1022B000B1F0878190850097A1F00E941505282F25
:1022C00092959F709630B9F080F4925F9F70923033
:1022D00030F4203FD1F058F481E0283E58F080E0FF
:1022E000089580819181D4DFEACF9A5FEFCF81E0BA
:1022F000243FA9F7089591E0813F09F090E081E043
:10230000283E08F080E0892B089581E00895382F59
:10231000292FCB01A32FB22F8F389105A105B1052D
:1023200020F48F589C4F0C94822E80E0089585E213
:1023300090E00E94822E8D3589F486E290E00E9422
:10234000822E8E3059F487E290E00E94822E91E036
:10235000853A09F090E0892F8170089580E0FCCFE4
:10236000AAE0B0E0E6EBF1E10C940F2EC090800201
:10237000D090810281E090E090938102809380026E
:10238000812C912C10E0540100E019C021E030E0D4
:10239000123020F4F701859195919C01472D602F13
:1023A000812FE2D9739422E0E20EF11C3FE0731218
:1023B000EDCF0F5F8FE0A80EB11C053049F0C501CD
:1023C000880F991FFC01E95DFC4F7F01712CDECF66
:1023D0001F5FFBE48F0E911C1430A9F61A8219823C
:1023E0001C821B821E821D8218861F8288EC90E050
:1023F0009A87898701E812E09E012F5F3F4F79019C
:102400004AE050E0B801C7010E94BC2E065F1F4F92
:10241000013D32E01307A1F78AE0F70111928A9596
:10242000E9F74AE050E0B801C7010E94BC2E065F00
:102430001F4F0132F3E01F07A1F789E0F701119266
:102440008A95E9F78FEF9FEF9E838D8387E08A87D8
:102450004AE050E0B801C7010E94BC2E065F1F4F42
:102460000137F3E01F07A1F7D0928102C0928002EA
:102470002A96EDE00C942B2EAAE0B0E0E2E4F2E123
:102480000C94142EE6EFF1E080E5DF011D928A95B1
:10249000E9F7E0E5F4E088E3DF011D928A95E9F7CA
:1024A00086EFC82E81E0D82E7F0101ED12E0F70102
:1024B000D182C0824AE050E0B801CE0101960E946C
:1024C000722E88E0FE013196D60101900D928A9518
:1024D000E1F789859A85D70113969C938E9312977D
:1024E000BAE0CB0ED11CE7E0EE0EF11C065F1F4FE9
:1024F0000132F3E01F07D9F62A96E8E00C94302E5B
:10250000AAE0B0E0E6E8F2E10C94122E0DE313E04D
:1025100081E2E82E83E0F82E97E0B92E25EFC22E57
:1025200021E0D22EAA24A3944AE050E0B701CE01C4
:1025300001960E94722EF8013896DF018B2D1D92B4
:102540008A95E9F789819A81D80111969C938E9397
:102550008F8112968C9312978D8113968C9313977B
:10256000888514968C931497898515968C93159766
:102570008B819C8117969C938E9316978A8587FDF5
:1025800004C01E96DC92CE921D9780FF02C0F80117
:10259000A08681FF07C0D80118969C911897926079
:1025A00018969C9382FF04C0F801908594609087F0
:1025B00083FF07C0D80118969C91189798601896C9
:1025C0009C9384FF04C0F80190859061908785FFFB
:1025D00007C0D80118968C911897806218968C9332
:1025E000BAE0EB0EF11C015F1F4FE1E7EE16E3E0EE
:1025F000FE0609F099CF2A96EAE00C942E2E282F99
:10260000CB01283070F44AE0249F90011124B901D5
:102610006F577D4F4AE050E00E94722E80E090E0BC
:1026200008958FEF9FEF0895AAE0B0E0EAE1F3E1AB
:102630000C941A2E9C0197558115914068F4BE01A7
:102640006F5F7F4F822FDBDF892B31F489859A857D
:102650002A96E2E00C94362E88EC90E0F9CFA0E0C8
:10266000B0E0E5E3F3E10C94152E162FD72FC42F1D
:10267000D22E8115A1F0409344040E94F00790935C
:10268000D8018093D701C77081E001C0880FCA9537
:10269000EAF7E5D8CDB7DEB7E7E00C94312E90919C
:1026A0004404491335C0E090D701F090D8010E944E
:1026B000F0079C012E193F097901812F9D2FB4DF6E
:1026C000E816F90628F5D0E2DD0DCD1591F0C770BA
:1026D00011E0812F01C0880FCA95EAF78AD9D83056
:1026E00040F48D2D877001C0110F8A95EAF7812F74
:1026F000B6D860E070E0802F66D9D83058F62D2D1E
:10270000277081E001C0880F2A95EAF772D9C2CFFD
:10271000C77081E001C0880FCA95EAF7F7CFA0E142
:10272000B0E0E5E9F3E10C940C2EFE01319680E176
:10273000DF011D928A95E9F709E010E091E7A92EE3
:1027400093E0B92E2FE8422E512C612C712C4F01B1
:1027500073016201B1E14B165104610471041CF074
:1027600080E1C82ED12CA601B501C4010E948F2E94
:10277000AC0CBD1C0D2C000CEE08FF084C185D08BD
:102780006E087F080150104019F76096E0E10C9444
:10279000282E6FEF85E290E00E949E2E6FEF86E27A
:1027A00090E00E949E2E6FEF87E290E00E949E2EA6
:1027B00060E088E290E00E949E2ED2DDB0DF6DE501
:1027C00085E290E00E949E2E6EE086E290E00E94FC
:1027D0009E2E65EA87E290E00C949E2EA0E0B0E089
:1027E000E4EFF3E10C94132EEC018881811509F1DB
:1027F000813009F045C08981813051F48A81239666
:1028000060E570E0893311F060E070E0DCD8EDCF76
:10281000823021F48A81239631D8E7CF833021F4A6
:102820008A812396A5D8E1CF843041F02296811188
:10283000DCCFCDB7DEB7E9E00C942F2E8A8123964A
:1028400020E030E09AE0682F6053770BAB016A30EC
:10285000710560F02115310551F3EFE9FFE0319783
:10286000F1F700C0000021503109F4CF929FB00170
:10287000939F700D11249A01260F371F8991E3CF82
:10288000E82FF0E0E850FE4FB490282F26952695CB
:10289000269530E0F901E851FE4FE4908770F12C65
:1028A000082E02C0F594E7940A94E2F7E0FAEE24C9
:1028B000FF24E0F8F901E852FE4FC490D12C082E15
:1028C00002C0D594C7940A94E2F7C0FACC24DD2460
:1028D000C0F8F901E853FE4F049110E002C01595CD
:1028E00007958A95E2F701701127E114F10419F0B8
:1028F00081EE0E943E0CC114D10419F086EE0E94B4
:102900003E0C60E070E08B2D5ED8C114D10411F054
:1029100086EE2ED8E114F10411F081EE29D80115CC
:10292000110521F060E070E08CE24DD821965DCF7A
:10293000ACE0B0E0EEE9F4E10C940B2E7C01DC019C
:1029400014968C91811509F4BDC161E0C7017EDC4C
:102950008C01F7018581811521F1809140049091CE
:1029600041040097F1F008171907D9F0FC01FF277F
:10297000887F9927892B09F072C0A4E0EE0FFF1F12
:10298000AA95E1F7E054FC4F85818460858311832B
:102990000083CF0167DB10924A0461E0C70156DC77
:1029A0008C01D70115968C91811509F4E1C0C801FD
:1029B00097578038910508F06AC1003108F071C15D
:1029C0006EE870E080E090E0A2DC81116AC1812CA9
:1029D000912C5401011146C004E09E012F5F3F4F2E
:1029E0006901D601E02F1D92EA95E9F7240135012E
:1029F000FFEF4F1A5F0A6F0A7F0AC501B40187DC37
:102A00008983811509F44DC1813009F0AEC0A5015B
:102A100094012E5F3F4F4F4F5F4F2D833E834F8377
:102A20005887C301B20173DC182F8A83811509F41A
:102A300038C18FEF810F833068F56D817E818F8182
:102A4000988565DC8B83811511F0C601C7DE2401F2
:102A5000350133E0430E511C611C711C49C0E0E09C
:102A6000F0E092CFBFE88B169104A104B10409F401
:102A700018C1C501B4014BDCEFEF8E1A9E0AAE0AF5
:102A8000BE0A8111EFCF0150A5CF4D805E806F80CF
:102A900078842EC08BEF810F833098F524013501A7
:102AA00043E0440E511C611C711C6D817E818F813D
:102AB00098852DDC8B838115D9F0C301B20127DC09
:102AC0008C83811571F08B819C8181305FEF95073C
:102AD00010F0982F8827163071F0173079F00E9487
:102AE000DD232401350134E0430E511C611C711CAF
:102AF0005301420176CF0E948A23F3CF0E94AB2379
:102B0000F0CF143009F0C1CF6D817E818F8198851F
:102B1000FEDB182F2401350184E0480E511C611C96
:102B2000711CC501B4016D5F7F4F8F4F9F4FEFDB6D
:102B3000111509F4B6C0811509F4B3C08150990B81
:102B40004FEF489F9001499F300D1124A12FA150B4
:102B5000BB0B2A0F3B1F2150310950F2EFE9FFE078
:102B60003197F1F700C00000F6CFC60137DEC0CFC5
:102B7000011527E5120708F4B9C0011538E5130758
:102B800008F0F8C7680147E5D41A6DE273E08C2DB0
:102B900036DD892B31F5C601E4E0880F991FEA95EF
:102BA000E1F7FC01E054FC4F2281213009F05BC0C9
:102BB00020912D0330912E03232B99F020912F0388
:102BC00030913003232B69F020913103309132038F
:102BD0004091330350913403242B352B232B09F4DC
:102BE0004CC080913703811509F404C1C09048049A
:102BF000D09047040E94F00788579C4E9093390369
:102C000080933803D70115968C91811509F4F2C091
:102C10008D2D8C298D7981111FC10115B0E51B0700
:102C200008F0BAC00115E0E41E0708F01CC1063E1A
:102C3000110509F4DFC0C80190528115904208F0D7
:102C400019C1D70116968C91803108F4FDC0C801D6
:102C5000992710924A048D32910509F0B6C082E09E
:102C600080934A040BC1223009F0BBCF209131037D
:102C700030913203232B09F4B4CFFC01EB53FC4F0A
:102C800020812E7F208380549C4FECD9AACF03371C
:102C90005CE7150759F5809137038115B9F00E945B
:102CA000090D80914B048770811561F0D70115964D
:102CB0008C91811539F08091020582FF03C082E07A
:102CC0000E94EE032C96E1E10C94272E109248040A
:102CD0000E9417040E94F00788579C4E9093390376
:102CE0008093380381E080933703DBCF023A82E59B
:102CF0001807C1F158F4C80190528115904220F193
:102D0000013E110579F1053E110503C0023BB2E514
:102D10001B0709F066CF25EE30E02770332781E0EE
:102D200090E001C0880F2A95EAF720913A0330918C
:102D300037033115F9F0D70115963C913115A9F0FB
:102D4000282B20933A03ADCFF7018681803108F01C
:102D500048CF812F99278F7199278230910511F0E3
:102D60004297D7CF21EE30E0D8CF80958223809351
:102D70003A0397CF322F3823311509F432CF982FE9
:102D80009095922390933A030E940F04F701858156
:102D9000811509F486CF25CF003EB2E51B0708F068
:102DA00046C0003CE2E51E0728F5003AF2E51F07A1
:102DB000E8F4003622E51207E8F4C80192558034A1
:102DC0009105C0F010924A04C8018E32910508F0B6
:102DD00062C08832910508F04FC08E31910508F02D
:102DE0004DC004974A9708F43ACF36C0043B32E509
:102DF000130741F7F7013580311409F456C00E3539
:102E0000FCE71F0709F44DC00F352CE7120751F0FE
:102E10000D353CE7130709F048C08091100181157A
:102E200009F43FC01092100180E041D93ACF093730
:102E30004CE7140728F407375CE71507D8F6C2CF2C
:102E40000B378CE71807D5CF812F8F71843191F222
:102E5000863111F410924A040E94090D80913A03C0
:102E60000E940904C7CFD70116968C91803108F0D3
:102E7000EECEC0CFC801EDCE8A9771F780913A03AC
:102E8000811531F080914A0492E0892780934A04A9
:102E90000E94DB0BAFCF8C34910581F38D329240D1
:102EA000ECCF81E080931001FCCE80911001811164
:102EB00069C0C80197558115914008F0FFC05801BD
:102EC000F8EFAF22BB24A114B10409F0EACEF80157
:102ED000FF2754E0EE0FFF1F5A95E1F79F012054A2
:102EE0003C4F6901D70115968C91EB53FC4F9081B3
:102EF00080FB90F99083811509F4D9C10E94F007F5
:102F00009093430480934204F60182818F5F828311
:102F100080914A0490914804892B838380914704CF
:102F200084834681578166857785C6010E9429077B
:102F3000D60115968C9181FF5801B0924104A09260
:102F40004004D70115969C91911509F42CC6109256
:102F50004404980130572332310508F00FC684E04D
:102F600090E00E948A2E9093020580930105F8015B
:102F7000E150F047E232F10508F0E1C1EE50F14DC9
:102F80000C94FD2D380150EE651A710850904904DB
:102F900080914804582A80914704582A88E068168E
:102FA000710408F05EC098012770332781E090E03B
:102FB00001C0880F2A95EAF7311409F44FC0582A46
:102FC000D7018D919C910E94910321E030E0F9019D
:102FD00002C0EE0FFF1F8A95E2F7FC87EB87209176
:102FE000B6033091B7033E832D834091BE035091C9
:102FF000BF035A8749876DE3C62E63E0D62EA12C06
:10300000B12C511005C0D60112968C9181111BC0B4
:10301000F601838190E02B853C8582239323892BC5
:1030200091F08085982F9770911101C087E038E06A
:103030006316710408F066C0311409F45FC0869508
:103040008170811164C09FEFA91AB90AAFE0CA0E5E
:10305000D11CB8E0AB16B104A1F61CC08095582273
:10306000AFCF311038C08091BE039091BF030817D5
:10307000190781F41092BF031092BE031092BA0395
:103080001092BB031092BC031092BD031092B903BF
:103090001092B8038091B6039091B703009709F49A
:1030A00008CFE8E06E16710408F0EBC0652D0E94B1
:1030B0008E06811103C081E00E945710F7018581BF
:1030C000F801E851FC47E730F10508F03ACFEC5E33
:1030D000F04D0C94FD2D1093BF030093BE030E948E
:1030E00047096093BA037093BB038093BC0390932A
:1030F000BD031092B9031092B80362CF82FB8827F8
:1031000080F99FCF311409F49ECF80FF9CCFD60168
:103110008D909C900815190519F4311409F493CF7A
:10312000ED81FE81EC15FD0509F48DCFD6011D96CC
:10313000ED91FC91309721F08081811509F483CFC6
:10314000652DC6010E948E06811509F47CCF81E0B1
:103150000815190509F080E0482E432081149104D8
:1031600041F0411006C0E985FA858E169F0609F0E8
:103170006ACF80E00E945710D092B703C092B60386
:1031800081E08093B5038FE08A9DF0018B9DF00D67
:103190001124E35CFC4F858180933C0341100EC0F9
:1031A0008114910459F0808191819C01245031094E
:1031B000213A310508F049C00E94C1078FE08A9D7D
:1031C000F0018B9DF00D1124E35CFC4FC680D7808D
:1031D000C6019A9581159F4110F420EED2229924C0
:1031E0009394C60101978F339E4708F0912C8FE08E
:1031F0008A9DD0018B9DB00D1124A35CBC4F199604
:10320000ED91FC911A97309731F01B966D917C915E
:1032100081E0099598229114A9F08FE08A9DF00130
:103220008B9DF00D1124E35CFC4F868197810E94F9
:10323000F70280933B03C60148E06416710440F432
:103240000E9453090E94DB0B0AC00E94B80CB6CF43
:103250000497813A910548F48C2D0E948D07411402
:1032600009F427CE0E94DB0B1CCD0E94DB0B8FE301
:103270009CE90197F1F700C000008C2D0E943E0CE4
:10328000EECFDC012D913C910217130741F4311070
:1032900009C01092B50380E00E9457100ACE311485
:1032A00009F407CEFC01808585FD03CEF4CFF9013A
:1032B0004485558566857785C9010E942907D60111
:1032C00015968C9181FF3DCEC6010E94161080910B
:1032D0004004909141040817190709F032CE10926A
:1032E0004104109240042DCE06E221EE41EE6AE147
:1032F0007CE7B5D9D6CC07E225EE45EE6BE17CE75D
:10330000F8CF06E221EE40EE68E17CE7F2CF07E27B
:1033100025EE44EE69E17CE7ECCF06E221EE42EED9
:103320006CE17CE7E6CF07E225EE46EE6DE17CE757
:10333000E0CF08E221E045EE6EE17CE7DACF809154
:10334000010581608093010560910105709102057E
:1033500084E090E00E94B82E0E94120DA2CC8091D1
:103360000205886080930205EFCF8091010582609D
:10337000E9CF809101058460E5CF809101058860E7
:10338000E1CF809102058160EDCF809102058260DE
:10339000E9CF809101058061D5CF809101058062E0
:1033A000D1CF809101058064CDCF0E94120D809114
:1033B00001058068C7CF809101058C60C3CF8091E3
:1033C00002058360CFCF809101058E7FBBCF8091B6
:1033D0000205877FC7CF809101058D7FB3CF809194
:1033E00001058B7FAFCF80910105877FABCF8091A7
:1033F00002058E7FB7CF809102058D7FB3CF80917C
:1034000001058F7E9FCF809101058F7D9BCF80919D
:1034100001058F7B97CF0E94120D809101058F7758
:1034200091CF80910105837F8DCF809102058C7FA4
:1034300099CF80910105992782FF939590FB82F99E
:1034400090FB83F97FCF80910205982F909590FB98
:1034500080F990FB81F986CF90910105892F8F7BB0
:1034600096FF80646FCF0E94120D90910105892F05
:1034700097FB87F9805866CF61E08EE090E00E946C
:103480009E2E62CF60E0F9CF90910105892F8F7E4B
:1034900094FF806157CF90910105892F8E7F90FF17
:1034A000816050CF90910205892F877F93FF8860BC
:1034B00059CF89E275C389E281C30737BCE71B078F
:1034C000F9F00837ECE71E0731F19801205E32452C
:1034D0002032310528F5911123C00F7181E090E071
:1034E0009C0102C0220F331F0A95E2F78901622F67
:1034F00083E090E00E949E2E802F0E943D03D1CB5E
:1035000081E0911551F00E94430343E062E081E0C5
:103510000E94C503C6CB82E0F4CF0E944D03F5CFD5
:103520004091460480910005282F30E02095309589
:1035300070E024233723232B19F0482340934604BB
:103540000B373CE7130741F4911509F4AACB0E940D
:103550002A030E94AF06A5CB003442E5140708F009
:1035600055C0003252E5150708F057C0011580E537
:10357000180750F50115A0E41A0708F064C091156A
:1035800009F479C00A35FCE71F0709F4CDC008F03B
:10359000B2C001303CE7130709F4C4C003304CE764
:1035A000140709F4B9C001151C4709F064C00E9452
:1035B000120DAFEFB4E3ECE0A150B040E040E1F712
:1035C00000C000000E94130B9801305521153240B5
:1035D000B0F6980145E0369527954A95E1F7822F98
:1035E0008F702091460430E041E050E0082E02C088
:1035F000440F551F0A94E2F724233523232B09F4A3
:10360000BECF9111A6CF109248042CCE9801205C19
:1036100032452032310508F0B2CF802F8F712091D2
:10362000460430E041E050E0082E02C0440F551F30
:103630000A94E2F724233523232B09F4A0CF911514
:1036400009F42FCB86CFF7018681803108F097CF20
:10365000911111C0212F2F7081E090E002C0880FDE
:10366000991F2A95E2F72091460430E082239323A4
:10367000892B09F016CBF70187819085009709F413
:1036800057C00E9415058C01F701B580A680A29451
:103690002FE0A22280914B048770811501F1CB2C81
:1036A000B114F1F0812F807F803461F080E2800FCF
:1036B0008830A8F0812F807E803221F4023078F0AB
:1036C000A11469F08091020582FF09C082E00E9486
:1036D000EE0380914B048770CC24C3948111C12CDC
:1036E000E12FE295EF70103C08F094C0F0E0E55E49
:1036F000F04D0C94FD2D0B358CE71807B9F0809137
:103700000205002482FF0394802D0C351C4709F02C
:10371000B2CF0E949E0BAFCF6FEF7FEF80E090E0C3
:103720000E94B82E0E943E0D81E0F3CF80E0F1CFE1
:103730008581C080D180811569F0C6010E94FC108E
:10374000182F682FC6010E945B03B601812F0E94CB
:10375000E11097CFC6010E949103182FF6CFF12FE9
:10376000FF70DF2E103118F0D29490EFD922B114EF
:10377000A9F0D11459F080E2800F883010F00111C7
:1037800007C08D2D0E9409040E94DB0B802F40C0D2
:1037900080914A048D2980934A04F6CF802F0E949D
:1037A000B80CD114B9F180E2800F883010F001110B
:1037B00004C08D2D0E940F0406C0D09480914A044D
:1037C0008D2180934A040E94DB0B24C0212F2F708F
:1037D000D22E107F103219F0D29480EFD82201152A
:1037E00049F0013009F482C0B11409F48EC0A1146B
:1037F000A1F1CCCF8091020582FD2BC0B11419F14B
:10380000D11429F08D2D0E9409040E94DB0B80E069
:103810000E943E0CC11409F4D8C080914B0480FD75
:10382000D4C0D70115961C928695869586950E94E0
:103830004303C7017DD880914B0486958695869574
:103840000E944D03C2C080E00E94B80CD11411F355
:10385000B0CFB11469F1A11004C08D2D0E942F0CBE
:10386000D9CF31E0A31210C0109147048D2D8123D0
:10387000D81681F20E94F00790934F0480934E0473
:103880001D2910934704C6CF45E0A412C3CF8D2D48
:103890000E942F0C8D2D0E944E08809149049D2D71
:1038A0009823D91609F4B6CF8D2980934904B2CF55
:1038B000A11012C08D2D0E94F90C8D2D0E944E0872
:1038C000809149049D2D9823911509F4A3CFD0949C
:1038D000D822D09249049ECF51E0A5129BCF80916F
:1038E00048048D21811509F495CFE4CFB11429F056
:1038F00086E0A81608F08ECFB0CF95E0A91608F0A4
:1039000089CF8D2D0E94F90C85CFA114D1F30933F5
:1039100049F4AFEFB7EEE3E0A150B040E040E1F78B
:1039200000C00000802F0E94B80C74CF812F8695B4
:1039300086958370811561F0813009F06BCFC801E5
:103940009370B11002C080E090E00E94650762CFE2
:10395000C8019370B11002C080E090E00E943D0762
:1039600059CF6B2D802F0E948C0854CF812F8370EC
:10397000811138C0B11027C0402F4295469547703D
:10398000440F440F802F8F70042E01C0880F0A94BB
:10399000EAF7202F207104FF07C02FE030E001C0BC
:1039A000220F4A95EAF72095169516951370123056
:1039B000A1F0133081F03091FF04113059F0822BC7
:1039C00083230E943D030E942E0760E0C7010E94EE
:1039D000261178C9832B822BF4CF822B9091FF0480
:1039E0008927EFCFB11451F110FFEDCF402F429551
:1039F00046954770440F440F802F8F70042E01C0EE
:103A0000880F0A94EAF7202F207104FF07C02FE0E7
:103A100030E001C0220F4A95EAF7209516951695D9
:103A20001370123089F0133069F0309100051130B5
:103A300041F0822B83230E944003C5CF823018F2CD
:103A4000D5CF832B822BF7CF822B9091000589272E
:103A5000F2CF1F70B11439F0812F0E944303802FE1
:103A60000E942F0CB0CF802F0E94F90C812F0E9452
:103A70004D03A9CF023F71F170F4003FC9F0013F3F
:103A800091F0B11409F465C0A11409F45FC0802F4E
:103A90000E943E0C98CF033F21F1043F91F78091A3
:103AA000020582FD2AC0812F8F71B11401F316C067
:103AB000B11469F0F5E0AF1608F085CF1F7181E011
:103AC00090E0012E01C0880F0A94EAF7BECF26E0ED
:103AD000A216F2CF812F8F71B110C9CF0E9443037C
:103AE00072CF80E0B11409F4A6CF1F7181E0012EDE
:103AF00001C0880F0A94EAF79ECFB114C1F08091FB
:103B00004B048770843049F410924B0410924D049A
:103B100010924C04812F8F71AACF35E063E0A31679
:103B200008F051CF812F8F710E943A084CCF45E0A9
:103B3000A41640F010924B0410924D0410924C04C5
:103B400064E0F0CF81E00E94EE033DCF812F8F71C2
:103B5000C5CFA114F9F2093349F45FEF87EE93E082
:103B6000515080409040E1F700C00000802F0E943B
:103B7000B80C29CF0337BCE71B070BC90631ECE7AC
:103B80001E0709F09ACC809148048A7A91E081114D
:103B900001C090E090934504811509F48ACC85E337
:103BA0000E948D075FCB0631FCE71F0709F085CC2B
:103BB00080914504811509F47ECC85E30E94C107FC
:103BC00051CBA0E0B0E0E7EEFDE10C94152E809122
:103BD0000303803108F049C080910203811509F484
:103BE00044C0C091B40289E0D82E8091B3028C17F2
:103BF000E1F1EC2EF12CDC9EE0011124FE01EB54EE
:103C0000FD4F84818115B1F191818091FE0298135D
:103C100031C090818091FD0298132CC08581811163
:103C200029C0028113818091FF0290910003081B3B
:103C3000190B60E08DEF92E00E9426110E94141390
:103C400008171907B8F4809103038F70806180937F
:103C50000303C554DD4F88818F70806188838DEFA9
:103C600092E00E9498140E94E403CDB7DEB7E7E02B
:103C70000C94312EE7012196C770B7CFAFE0B0E0CA
:103C8000E4E4FEE10C940D2E8C0186E0F801DE01E7
:103C90001A9601900D928A95E1F7F801F580E4807B
:103CA0008DEF882E82E0982E80910103811117C03C
:103CB000E11491F0F11409F480C1C8010E9455117A
:103CC000811509F47AC189E0F801ADEFB2E0019005
:103CD0000D928A95E1F775DFFF24F3946AC0A28004
:103CE000B380D09002038091FF02909100033501D0
:103CF000681A790AD11409F411C1C080518060E0BA
:103D00008DEF92E00E9426110E9414136816790626
:103D100008F0B6C0E11401F38091FE02F801918130
:103D2000E0900303F0E1EF1608F064C0981320C0A0
:103D30009091FD02F801808198131AC0209104032C
:103D400030910503878190852817390789F4F11090
:103D50004BC08E2D8F708061809303038DEF92E0B6
:103D60000E94981480910303F8018683F12C21C0EE
:103D7000F1103AC040E0652D8C2D0E94F40A40E01D
:103D8000652D8C2D0E94F40AF82E8111EFCF8A85C3
:103D90009B850E944811292F22952F70903470F432
:103DA0009F702230A0F09115B1F0F801968190310A
:103DB00090F48F2D2F96EFE00C94292E2A5F2F7010
:103DC000223068F0C8010E949814FD2CF2CF9115A2
:103DD00011F0811571F3805E883058F3F3CF803F86
:103DE00040F3815F8330F9CF80910303816080933A
:103DF0000303BCCF98131EC09091FD02F80180818F
:103E0000981318C020910403309105038781908591
:103E10002817390779F4F1100DC0E682C8010E9415
:103E2000981489E0F801ADEFB2E001900D928A9507
:103E3000E1F752CFC8010E945511811509F4BDC0A8
:103E4000F11409F4BAC080910303803208F43BCF27
:103E50008091FD029091FE029A838983BC82AB829D
:103E6000809101038D831E82EF82809104039091E3
:103E7000050399878887CE0101960E94981423CF65
:103E8000D0900303F0E1DF1650F48DEF92E00E9432
:103E9000981489E0F40111928A95E9F767CFE1144B
:103EA00009F41ACF9091FE02F801818198131AC08B
:103EB0009091FD028081981315C0209104033091E8
:103EC0000503878190852817390761F4F1100AC02E
:103ED000D682C8010E94981489E0F40111928A9553
:103EE000E9F7FACEC8010E945511811509F465C0A1
:103EF000F11409F462C080910303803208F4E3CE28
:103F00008091FD029091FE029A838983BC82AB82EC
:103F1000809101038D831E82DF82A7CF60E08DEF49
:103F200092E00E9426110E9414136816790608F088
:103F3000B0CFE11409F4D0CEF11409F43EC0909151
:103F4000FE02F801818198132EC09091FD028081BC
:103F5000981329C02091040330910503878190852F
:103F60002817390701F58091FF0290910003A81AE4
:103F7000B90AF8ECAF16B10408F053CF80910303EF
:103F800080FD4FCF803108F44CCFF8018683982F05
:103F9000907F903F09F442CF982F907F905F8F7071
:103FA000892B86833BCFC8010E94551181118BCE8E
:103FB00080910303816080930303C8010E949814D9
:103FC0008BCEA2E1B0E0E7EEFFE10C94182E0A8759
:103FD0001B872C873D874E875F87688B798B8A8B01
:103FE000CE010A964BDE811128C02091B302309198
:103FF000B40289E0FE013A96DE01119601900D921D
:104000008A95E1F78E858115C1F0822F90E00196A7
:104010008770992738171906D9F099E0929FD00137
:104020001124AB54BD4FFE01319601900D929A952B
:10403000E1F78093B3020E94E40319E08091B40297
:104040009091B302891312C06296E4E00C94342E6E
:104050000E94120D1092B3021092B40289E0EDEFAB
:10406000F2E0DF011D928A95E9F7E7CF189FC001C2
:1040700011248B549D4F02DE811531F38091B402DF
:1040800090E00196877099278093B402D7CFEF9282
:10409000FF920F931F93CF93DF938091FC04E091E5
:1040A000F401CDE0811130C0CDB7DEB7E6E00C946D
:1040B000322ED1E0DE0FD093F401EE2EF12CCE9F04
:1040C000F0011124EC56FB4F84818115E1F08781CA
:1040D0009085892B21F481859285019651F4008188
:1040E0001181228133814481558166817781808568
:1040F00068DFCE9DF001CF9DF00D1124EC56FB4FF3
:10410000148210924A04ED2F8091FC04E81788F283
:104110001092FC041092F401C7CFA4E0B0E0E3E9F0
:10412000F0E20C940B2E20919304298397E0992EB2
:1041300001E010E02DE0322E34E0532E88248394E9
:10414000809192049981891307C0A1DF0E945106D2
:104150002496E1E10C94272E9981892F90E09C838D
:104160008B83FC01EE0FFF1FE857FB4F808191818D
:10417000989ED001999EB00D1124FD01E05BFB4F8C
:10418000FA83E983248121115BC06090FC04E4E997
:10419000F4E060E070E0712C661508F04FC0A38475
:1041A000B484A981BA81CD90DC902FEF3FEF412CF0
:1041B000442D50E07601E40CF11CE40CF11CD70115
:1041C000ED90FC90E114F10439F0AE14BF0409F055
:1041D000A90143949A01ECCF2F3F3207D1F1D801C6
:1041E00002C0AA0FBB1F2A95E2F77A2A9801042C75
:1041F00002C0220F331F0A94E2F7A901415051096E
:104200007416150629F5369EF001379EF00D11241F
:10421000EC56FB4F989ED001999EB00D1124A05BE7
:10422000BB4F12962D913C91139730872783548270
:10423000108211829287818715968C920E94620665
:104240008B819C8101969A8389838370898378CF3F
:1042500014826F5F7F4F3D969FCF1092FE041092A5
:10426000FD041092110180919204809393040E94A6
:1042700051060DCFACE1B0E0E0E4F1E20C940A2E7F
:104280004B8B5C8B6D8B7E8B8F8BB92E988FA92E71
:10429000911110924A04188A198A1A8A86E0FE013E
:1042A0007396DE011A9601900D928A95E1F75F8868
:1042B0008091020582FF1FC00E94F00720914C04EC
:1042C00030914D04821B930B8838934138F08091D4
:1042D0004B0482FD03C082E00E94EE030E94F007BF
:1042E00020914E0430914F04821B930B88389341E8
:1042F00010F00E9417045114D9F05E86BF8661E069
:10430000CE010A960E94261161E0CE010A960E9413
:10431000261161E0CE010A960E9426114C018035DB
:104320006CE7960791F4A11419F181E080931101D3
:104330005E86BF860A851B852C853D85452D5B2DB8
:10434000688979898A893DDECDC081359C4721F411
:10435000A11471F082DFECCF82E588168CE7980615
:1043600039F4A11429F0809111018111F3CFDDCF2F
:1043700040E5E42E44E0F42E412C612C712CD70151
:104380006D917C91CC24CA94DD24DA9480E0282FAE
:1043900030E0FB01E80FF11DE80FF11D4081518174
:1043A0004115510539F08416950609F096018F5F85
:1043B0006901EDCF10E0BFEFCB16DB0609F44EC06C
:1043C000F701448110911101411110E0D7011596B8
:1043D0003C90159716969C911697A11409F405C167
:1043E000111509F402C1311017C021E030E00C2C86
:1043F00001C0220F0A94EAF7922B16969C93209103
:104400009004309191042233310530F422E330E0FE
:104410003093910420939004E1E0F0E002C0EE0FAD
:10442000FF1F8A95E2F7CF010197D70116962C91CD
:104430002817190699F4C090FD04D090FE04C11409
:10444000D10409F453C00E94F0078C199D09C39749
:1044500008F44CC081E0F701848311E0412ABFEFEA
:104460006B1A7B0AE7E0EE0EF11CF8E06F167104A0
:1044700009F085CFA11409F417C1411409F414C13E
:104480000E94F0079093FE048093FD048091FC0449
:10449000883040F591E0980F9093FC0499E0FE017C
:1044A0003A96DE01119601900D929A95E1F75D82A0
:1044B000BE822DE0829FC00111248C569B4F29E0C3
:1044C000FE013196DC0101900D922A95E1F72FEF64
:1044D0003FEFDC011A963C932E9319971C969C9201
:1044E0008E921B976C96E2E10C94262E20919304F9
:1044F00080919204922FE0E0F0E001E0281709F4A7
:1045000048C0422F50E0FA01EE0FFF1FE857FB4F63
:104510002080318037E0329DF001339DF00D112471
:10452000E05BFB4F608171817C8F6B8FB0E030E08E
:10453000A0E0EB8DFC8DEA0FF11DEA0FF11DC080AC
:10454000D180C114D104E1F0F7010190F081E02D98
:10455000FA8FE98F30E007C0E1E0C616D70609F010
:10456000E0E0BE2B3F5FE98DFA8DE30FF11DE30F15
:10457000F11D608171816115710571F7AF5FD9CF50
:10458000B11581F13A17C8F4E1E0D7011496EC9324
:10459000F70190939304EE15FF0509F45FCF90E0C7
:1045A000FC01EE0FFF1FE857FB4F718260820196FE
:1045B000837099278093920451CF37E0329DF001A8
:1045C000339DF00D1124E05BFB4F0483EE15FF05D6
:1045D000F9F2291302C09F5F93709A012F5F3F4F3A
:1045E00023708CCFE0E0F0E0F8CF292F30E03110DD
:1045F00024C061E070E002C0660F771F8A95E2F781
:10460000CB0101972817390791F010E0E1E0F0E0C5
:1046100002C0EE0FFF1FCA94E2F76F01C094D701EA
:1046200016968C9116978C2116968C9317CF411560
:1046300069F3C3010E946206E8CFA9010C2C02C0F5
:10464000559547950A94E2F7C90101978223932370
:10465000892B39F540FF25C0D70112968D919C9189
:10466000892BD1F087E0FE013196DF011D928A95FA
:10467000E9F70E94F0079C018B839C8384E08D8383
:10468000F70192818381792F9887898709811A811F
:1046900044E05E816F8195DCD70115961C92132D45
:1046A000B5CF142F1170B2CF9091930480919204E2
:1046B000981731F032DDB1E04B1609F413CF38CE44
:1046C000E6DC1092FE041092FD040E945106F3CF26
:1046D000A6E0B0E0EEE6F3E20C94182E0E94F0079C
:1046E0008C0180918702909188028017910771F068
:1046F00019821A820E94F007BC0149815A8180E028
:1047000090E0B8DD10938802009387022696E4E0DB
:104710000C94342EA6E0B0E0E0E9F3E20C941A2EFB
:104720009093840280938302811520E2920730F4F3
:104730000E94A30C2696E2E00C94362E80EF89832B
:104740008A830E94F0078160BC0149815A8181E01F
:1047500091E090DDEFCFA6E0B0E0E1EBF3E20C9466
:10476000182E8C019093840280938302011580E2BD
:104770001807B0F4802F0E94B80CC801805E910920
:10478000089728F06FEF7CE00115110511F469EF2F
:104790007CE0C8010E9421032696E4E00C94342EAC
:1047A00080EF89838A830E94F0078160BC01498180
:1047B0005A8181E090E05EDDEFCFCF93DF93D82F79
:1047C000C92FA8DF8D2F9C2FC6DFDF91CF910895D1
:1047D0000F931F93CF93DF938C01862F6DE273E0CD
:1047E0000E94FF12892B91F4C0912D03D0912E03CA
:1047F000209761F0F8018281833039F4CE01DDDF4A
:10480000CE01DBDFCE01D9DF01C0E0F7DF91CF9130
:104810001F910F9108950F931F93CF93DF938C01F6
:10482000EB016DE273E08C2F0E94FF12892B09F0DF
:1048300057C0FE01FF27D80112968C911297EA5BB0
:10484000FD4F8130A9F415968C9182FD4EC080FFFA
:104850004CC082E0808380912F03909130030097B9
:10486000B9F480912D0390912E030097C9F110C0E7
:104870008230A1F515968C9182FD26C080FD0AC07C
:1048800083E0808380913103909132030097F1F0AF
:1048900041DF26C084E0808380913303909134030C
:1048A0000097B1F780912D0390912E03009701F1AD
:1048B00084DF80912F0390913003009749F7809116
:1048C0002D0390912E03E4CF85E0808380912D030A
:1048D00090912E03009721F070DFF1CF86E0808366
:1048E000DF91CF911F910F91089581E08083B9CF1F
:1048F00080912F0390913003B8CF0F931F93CF93E4
:10490000DF938C01EB016DE273E08C2F0E94FF12AC
:10491000892B71F4DD27CA5BDD4F8881F801128293
:1049200018828330E9F048F4813059F0823081F008
:10493000DF91CF911F910F9108958430B1F08530B0
:10494000B9F780912D0390912E03009789F306C04B
:1049500080912F0390913003009799F3FCDEE8CF0C
:104960008091310390913203F7CF8091330390917E
:104970003403009799F720912D0330912E038091F5
:104980002F039091300321153105F9F2009731F78B
:10499000C901E4CFAAE0B0E0E0EDF4E20C940E2E01
:1049A000FE0131968AE0DF011D928A95E9F79AE2CD
:1049B000A92E91E0B92E8F013F01EE24E394F12C52
:1049C0003EE3C32E31E0D32EF50181915F018F3F8D
:1049D00009F444C0F894E82FE295EF70F0E021A1CB
:1049E0008F70A70102C0440F551F8A95E2F7CA01D4
:1049F000922F982B91A392A18095892382A37894DA
:104A000000C0EFE2F1E021E030E0812C912C4191F7
:104A10004F3F79F0A42FA295AF70A05EB0E08C91CB
:104A200090E04F7002C0959587954A95E2F780FF18
:104A30003BC080E090E0882A992A220F331FCE16CF
:104A4000DF0629F7F50182918F3F11F00E941306CE
:104A500050EA5A95F1F7D8018D929C920E5F1F4F44
:104A6000BFE2AB16B1E0BB0609F0AECF4AE050E0C2
:104A7000B3018EE492E00E945E2E892BB9F08AE0A9
:104A8000F301AEE4B2E001900D928A95E1F781E086
:104A90008093D6010E94F0079093D5018093D401B2
:104AA0002A96EEE00C942A2EC901C5CF8091D6013A
:104AB0008115B1F30091D4011091D5010E94F00746
:104AC000801B910B059760F34AE050E06EE472E0C2
:104AD00086E792E00E945E2E892B49F08AE0EEE4A0
:104AE000F2E0A6E7B2E001900D928A95E1F710920C
:104AF000D601D6CFCDB7DEB7AC970FB6F894DEBFF0
:104B00000FBECDBF85B7806885BF85B7806885BF7C
:104B100084B7877F84BF0FB6F894A8958091600012
:104B2000886180936000109260000FBE80E890E082
:104B30000FB6F89480936100909361000FBE81E0FE
:104B400080930F0181E196E09093AB018093AA01DD
:104B50000E9439060E943C120E9480120E943D0A67
:104B60000E949A0A8091E20084608093E200789427
:104B700080918202811599F08091E9001091EC00FA
:104B80008F70179511271795182B1092E9008091B7
:104B9000E80083FD0E94530D1F701093E90082E02E
:104BA00084BD93E095BD9AEF97BD80936E000E94FF
:104BB0009711811102C00E94C9130AE211E0D801C5
:104BC0008D918D018F3F11F00E941306B1E00F32DD
:104BD0001B07A9F70FE211E0F80181918F018F3FC8
:104BE00011F00E941306F1E00E331F07A9F78AE0C7
:104BF000E6E7F2E0DF01282F1D922A95E9F7EEE4BF
:104C0000F2E0DF011D928A95E9F780E090E00E94D2
:104C10008A2E833E9E4F21F40E949711811129C054
:104C200063EE7EEF80E090E00E94B82E60E082E0CC
:104C300090E00E949E2E81E08093FF0461E083E07B
:104C400090E00E949E2E60E074E184E090E00E947B
:104C5000B82E0E94C91340E050E0BA018FE090E006
:104C60000E94B02E40E050E0BA0183E190E00E9443
:104C7000B02E82E090E00E94822E80935A0284E05F
:104C800090E00E948A2E909302058093010582DEB7
:104C9000EFEFF6E721E0E150F0402040E1F700C0FF
:104CA000000078DE8091760280FF08C06FEF7FEF12
:104CB00080E090E00E94B82E0E94130B83E090E009
:104CC0000E94822E0E943D0380E091E09093AA0210
:104CD0008093A90280918202853049F480918202FA
:104CE000853009F45AC00E94120D0E942E0752DE30
:104CF000EBE5AE2EE2E0BE2E06E712E0D801F501AC
:104D0000219131918D919D9142E0E536F40709F4AE
:104D100079C028173907A1F376E7872E72E0972E1E
:104D2000512CD401ED90FD904D01F50161907190F1
:104D30005F016E147F0451F16E247F24412CCC243A
:104D4000C394D12CC3018C219D21892BB1F04982C0
:104D50005A820E94F0079C838B83F1E0FD8391E0EF
:104D600097012C213D21232B09F490E09E8349815A
:104D70005A816B817C818D817DDA4394CC0CDD1C62
:104D80002FE04212DFCFF501F292E292539435E028
:104D90005312C7CF0E9447093AC0809182028430E3
:104DA00021F11092580288E190E0A0E40FB6F89447
:104DB000A895809360000FBEA093600083B7817FA9
:104DC000846083BF83B7816083BF7894889583B7FD
:104DD0008E7F83BF0FB6F894A8958091600088619C
:104DE00080936000109260000FBED4DDE6E7F2E031
:104DF00081919191892B09F052C5B2E0E038FB070F
:104E0000B9F76CCF2817390709F086CF61DCE0903D
:104E1000B803F090B903E114F10491F180906902B4
:104E200090906A02A0906B02B0906C020E944709B9
:104E3000681979098A099B09809065029090660239
:104E4000A0906702B0906802681579058A059B05F5
:104E5000B8F0C7010E94A30C1092B9031092B803D6
:104E60001092690210926A0210926B0210926C0208
:104E70001092650210926602109267021092680208
:104E8000C0904004D0904104C114D10439F1A090E5
:104E90004204B09043040E94F0077C01EA18FB082A
:104EA000C6010E9414138E159F05C0F42091400482
:104EB00030914104C9019927287F3327232B09F01A
:104EC00055C144E0880F991F4A95E1F780549C4FE3
:104ED000DC0115962C9122FF0E9432108091110165
:104EE000811511F1E090FD04F090FE04E114F1044D
:104EF000D9F00E94F0078E199F09209190043091FB
:104F000091042817390780F49091930480919204BA
:104F1000981709F42EC101D91092910410929004AF
:104F20001092FE041092FD0480913703811569F000
:104F30000E94F0072091380330913903821B930BB4
:104F40008F3F9F4710F40E94090D86E0E7E2F3E0EF
:104F5000DE01119601900D928A95E1F79090280359
:104F6000B0902903D0902A03A0902B03C0902C036B
:104F70001092290310922A0310922B0310922C03F3
:104F80008D2D8B29811509F441C0E0906F02F090BE
:104F900070020E94F0079C012E193F099091250391
:104FA000911509F477C42531310580F19F3F19F03F
:104FB0009F5F90932503B11459F00E94E40691E09D
:104FC0001B140CF09FEF899F802D112480932903DF
:104FD000D11459F00E94E40691E01D140CF09FEFEB
:104FE000899F802D112480932A03809129038115A4
:104FF00069F0F0902A03F11449F00E94D6068093DC
:1050000029038F2D0E94D60680932A038A2D8C298E
:10501000811509F441C0E0906D02F0906E020E948B
:10502000F0079C012E193F0990912403911509F472
:105030002CC42135310580F19F3F19F09F5F90937B
:105040002403A11459F00E94040791E01A140CF0F3
:105050009FEF899F802D112480932B03C11459F059
:105060000E94040791E01C140CF09FEF899F802D93
:10507000112480932C0380912B03811569F0F0900B
:105080002C03F11449F00E94D60680932B038F2D38
:105090000E94D60680932C0380912803891119C0A1
:1050A00080912903811511F08B1113C020912A03DF
:1050B000211511F02D110DC090912C03911511F0B7
:1050C0009C1107C030912B03311103C0822B892B17
:1050D00081110E94630886E0FE013196A7E2B3E0E9
:1050E00001900D928A95E1F70E942E07909171022E
:1050F000891721F0809371020E94470980918202F2
:10510000843009F0E7CD83E08093E9008091E800E6
:1051100082FFE0CD8091E80090E085FF05C00E940D
:105120000C0A811579F191E08091E8008B778093EA
:10513000E800911509F4CECDE0908502F09086024A
:10514000E981E114F104E1F1EE3F09F05CC08A81EC
:10515000833020F08550833008F055C0EA81EE306E
:1051600008F051C0F0E0E95DF04D47C580E090E007
:10517000AFCE0E9447201092FE041092FD040E94C0
:105180005106D2CE30E2E32EF12CFE0131966F01B2
:105190008091E80085FD0AC08091E8008B778093BC
:1051A000E8000E940C0A811599F3BDCF8091F100AF
:1051B000D6018D936D01B1E0EB1AF10849F7B3CF39
:1051C000E43148F4E11551F0E150E33138F4F0E016
:1051D000EB5CF04D12C5EE3F09F4C0CFEFEFE98371
:1051E00012C01A8289E08B830EC08A81823081F0DE
:1051F0008330B1F0813091F70E94470904D56B8369
:105200007C838D839E83CE0101960E945C0A62CDD1
:1052100088E290E077D51B821C821D828E83F3CFBB
:105220008091800290918102892B69F3FE01319671
:10523000D8018C9111969C910E5F1F4F92838383AE
:105240003296B2E000381B0799F7DDCF8A818230B1
:1052500049F46B817C818D819E81D5D488E290E078
:105260006DD5D1CF8FEF8983CECF4C816B818A8171
:105270000E94B2109827892798279E838D83C3CFD9
:105280002D813E813227232732274C816B818A81F1
:105290000E94B40BB8CF0E94B011B5CF80E18A83D1
:1052A000B2CF1A828FE89FCF8C818D3108F0ABCFBF
:1052B0008A809B80982489249824A12CB12C9E015B
:1052C0002F5F3F4F79018901080F111D0E151F0532
:1052D00009F499CF80E03FE883169104A104B1045A
:1052E00020F4C4018F589C4F0DD5D70114968C9390
:1052F000BFEFEB1AFB0AEFEF8E1A9E0AAE0ABE0A48
:10530000E5CF8091800290918102892B09F47BCFB7
:105310008C818D3108F077CF882E912CA12CB12C67
:10532000CA80DB80DC24CD24DC24E12CF12C8E012E
:105330000F5F1F4F412C512C3201481459046A044D
:105340007B0408F060CFFFE8CF16D104E104F1043C
:1053500038F4D80114966C91C6018F589C4FEED446
:10536000BFEF4B1A5B0A6B0A7B0AEFEFCE1ADE0A1D
:10537000EE0AFE0A0F5F1F4FE0CF0E948F1343CF4C
:1053800084E08DCF8C818D3108F03DCF882E912C1B
:10539000A12CB12CCA80DB80DC24CD24DC24E12CC0
:1053A000F12C412C512C32018E010B5F1F4F481400
:1053B00059046A047B0408F026CF80E0F8E5CF1694
:1053C000F2E0DF06E104F10418F4C60189969AD4EC
:1053D000D8018D938D01BFEF4B1A5B0A6B0A7B0AD4
:1053E000EFEFCE1ADE0AEE0AFE0AE1CF2C81022F81
:1053F00010E02D3108F007CF8A819B8198278927FB
:1054000098272C01612C712C8835F2E09F0708F059
:10541000FACE822E912CA12CB12C48E552E060E00E
:1054200070E044195509660977094217510561056D
:10543000710508F4E8CE2091800230918102232B7F
:1054400009F03EC01C0129E2220E311C80FBEE2433
:10545000FF24E0F880FF0BC0889654D49D818927F3
:105460009827892781159C4711F48FEF8D83D501EB
:10547000C401840D951DA61DB71D80FF19C06801CC
:1054800041E0C41AD108CE0105968C0D9D1D9CA744
:105490008BA7C101800F911F35D4ABA5BCA59C91F2
:1054A00081159C4721F48FEFEBA5FCA58083860135
:1054B000FE013196EE0DFF1D2FEFE016F10638F0DC
:1054C0008E010F5F1F4FC12CD12C760125C0948116
:1054D000858181159C4711F42483258342E0E40EE5
:1054E000F11C3296EACF88E5481682E0580661043E
:1054F000710430F4D80114966C91C20189961ED4BF
:10550000BFEFCB1ADB0AEB0AFB0AEFEF4E1A5E0A7B
:105510006E0A7E0A0F5F1F4FC814D904EA04FB0409
:1055200010F371CE8091800290918102892B09F451
:105530006ACECE0101960E945C0AFFEF21EE34E0B4
:10554000F15020403040E1F700C00000B5CB88E0CA
:10555000E2E1F1E0DE01919601900D928A95E1F78A
:10556000FE0132968FE1DF011D928A95E9F786E010
:10557000898388E07F96DE01159601900D928A95C9
:10558000E1F741CE88E2898381E08A831B821C8215
:105590003ACE8B819C81092E000CAA0BBB0B25E017
:1055A000880F991FAA1FBB1F2A95D1F7AC01BD0117
:1055B000405E5F4F6F4F7F4F481759076A077B0761
:1055C00008F421CE8832E1E09E07A105B10508F07C
:1055D0001ACE4932F1E05F076105710520F048E21B
:1055E00051E060E070E0481B590BBC016D5A7B4FE5
:1055F000CE0101965AD307CE4AE150E06FEF70E03A
:10560000CE01079668D3809180028983EA821B824B
:105610001C8282E08D838CE001CE81E090E090934B
:1056200086028093850282E390E0909375028093D6
:1056300074020E94F0079093730280937202E3CD8C
:10564000E114F10481F1D0907602C0907B020091C8
:105650007202109173020E94F007801B910B853635
:10566000910540F1C4FE26C0D0FE24C00E94F00780
:1056700090937302809372028091740290917502EC
:1056800001979093750280937402892B61F41092B4
:1056900086021092850281E090E0909381028093CF
:1056A0008002E12CF12C809180028983EA82809132
:1056B000740299CD82E390E0909375028093740216
:1056C000F2CF10928102109280029DCD40E250E014
:1056D0006FEF70E0CE010196FED295CDEB81E73001
:1056E00008F091CDF0E0E85BF04D87C2FE01349602
:1056F0008CE1DF011D928A95E9F788E089838A832E
:105700008B8383E088A37FCD8C819AE0F92E8E0174
:105710000F5D1F4FF8012F2D11922A95E9F7B8015F
:105720000E94FF128983F801DE01129601900D920A
:10573000FA94E1F768CD1C818AE0FE013596DE011E
:10574000919601900D928A95E1F789A19AA10E9404
:105750002C069AA389A38BA19CA10E942C069CA332
:105760008BA38DA19EA10E942C069EA38DA38FA129
:1057700098A50E942C0698A78FA38FEF183060F48D
:105780003AE0139FB00111246F577D4F4AE050E07B
:10579000CE018196F1D280E089830E94390633CD13
:1057A0002C816AE0CE018196DC01E62F1D92EA95FC
:1057B000E9F7283008F044C0629FB00111246F520D
:1057C0007D4F4AE050E08ED280E089838AE0FE017E
:1057D000B196DE011296D1CE1C818AE0FE0135968B
:1057E000DE01919601900D928A95E1F789A59AA51F
:1057F0000E942C069AA789A78FEF183060F4FAE070
:105800001F9FB00111246F527D4F4AE050E0CE013E
:105810008196B2D280E089830E943C12F4CC2C8124
:105820006AE0CE018196DC01E62F1D92EA95E9F748
:10583000283030F4629FB00111246F5D7C4FC1CFDE
:105840008FEFC3CF1C818AE0FE013596DE01919671
:1058500001900D928A95E1F78BA19CA10E942C06E4
:105860009CA38BA38FEF183060F4FAE01F9FB00168
:1058700011246F5D7C4F4AE050E0CE0181967CD2CE
:1058800080E089830E948012BECC2B30310508F065
:10589000D5CB02CC2B30310508F08ACBB7CB809129
:1058A0005902811509F41ACAE0E1E9BDF2E1F9BD36
:1058B00009B400FEFDCF8091D8008F7D8093D80081
:1058C0008091E00082608093E0008091E00081FDA3
:1058D000FCCF0E94120D02CA1F921FB61F92112404
:1058E0008F939F93AF93BF9380915802811113C000
:1058F0008091EC019091ED01A091EE01B091EF014A
:105900004196A11DB11D8093EC019093ED01A093F0
:10591000EE01B093EF01BF91AF919F918F911F90D6
:105920001FBE1F90189578941F921FB61F921124C6
:105930008F939F93AF93BF938091EC019091ED0172
:10594000A091EE01B091EF010196A11DB11D8093D0
:10595000EC019093ED01A093EE01B093EF01BF91A4
:10596000AF919F918F911F901FBE1F9018951F920E
:105970000F920FB60F9211242F933F934F935F9383
:105980006F937F938F939F93AF93BF93EF93FF9307
:105990008091E10082FF09C08091E20082FF05C092
:1059A0008091E1008B7F8093E1008091DA0080FF9D
:1059B00024C08091D80080FF20C08091DA008E7FC3
:1059C0008093DA008091D90080FFA9C080E189BD71
:1059D00082E189BD09B400FEFDCF81E0809382029F
:1059E0008091DB01811109C00E943D0A0E949A0A40
:1059F0008091E20084608093E2008091E10080FF6A
:105A00001AC08091E20080FF16C08091E2008E7F74
:105A10008093E2008091E20080618093E2008091B7
:105A2000D80080628093D80019BC85E08093820200
:105A300083E080930F018091E10084FF2FC080916B
:105A4000E20084FF2BC080E189BD82E189BD09B4F9
:105A500000FEFDCF8091D8008F7D8093D80080918B
:105A6000E1008F7E8093E1008091E2008F7E809341
:105A7000E2008091E20081608093E2008091DA018F
:105A8000811509F452C084E08093820280918202E1
:105A9000843009F052C082E080930F018091E100D0
:105AA00083FF2CC08091E20083FF28C08091E10039
:105AB000877F8093E10082E0809382021092DA0176
:105AC0008091E1008E7F8093E1008091E2008E7FE3
:105AD0008093E2008091E20080618093E20042E0E6
:105AE00060E080E00E946A0A8091F0008860809304
:105AF000F00081E080930F0180930E01FF91EF9100
:105B0000BF91AF919F918F917F916F915F914F91D5
:105B10003F912F910F900FBE0F901F90189519BCB9
:105B2000109282021092DB0168CF8091E30087FF20
:105B300002C083E0A9CF81E0A7CF81E0ADCF1F9263
:105B40000F920FB60F921124EF92FF920F931F93B3
:105B50002F933F934F935F936F937F938F939F9375
:105B6000AF93BF93CF93EF93FF9309EE10E0F8014B
:105B70008081C091EC008F70C795CC27C795C82B4A
:105B8000108280EFE82EF12CF7018081877F8083DF
:105B900078940E94530DF8011082F701808188608B
:105BA0008083CF70F801C083FF91EF91CF91BF91B7
:105BB000AF919F918F917F916F915F914F913F91A5
:105BC0002F911F910F91FF90EF900F900FBE0F90AC
:105BD0001F90189597FB072E16F4009406D077FDBA
:105BE00008D04FD007FC05D03EF4909581959F4F8B
:105BF0000895709561957F4F0895EE0FFF1F0590F2
:105C0000F491E02D0994692796276927782787273B
:105C1000782708952F923F924F925F926F927F92D2
:105C20008F929F92AF92BF92CF92DF92EF92FF92AC
:105C30000F931F93CF93DF93CDB7DEB7CA1BDB0B58
:105C40000FB6F894DEBF0FBECDBF09942A883988FD
:105C500048885F846E847D848C849B84AA84B98404
:105C6000C884DF80EE80FD800C811B81AA81B98110
:105C7000CE0FD11D0FB6F894DEBF0FBECDBFED0124
:105C80000895AA1BBB1B51E107C0AA1FBB1FA61783
:105C9000B70710F0A61BB70B881F991F5A95A9F7D5
:105CA00080959095BC01CD010895FB01DC0102C0F7
:105CB00005900D9241505040D8F70895FB01DC014A
:105CC00004C08D910190801921F441505040C8F7D3
:105CD000881B990B0895DC0101C06D934150504021
:105CE000E0F70895DC01CB01FC01F999FECF06C075
:105CF000F2BDE1BDF89A319600B40D92415050408A
:105D0000B8F70895F999FECF92BD81BDF89A992709
:105D100080B50895A8E1B0E042E050E0E5CFDC01B5
:105D2000A40FB51F4150504040F0CB01840F951F88
:105D30002E9105D041505040D8F70895262FF9995B
:105D4000FECF92BD81BDF89A019700B4021639F0DA
:105D50001FBA20BD0FB6F894FA9AF99A0FBE0895AB
:105D60000396272FECDFEADF252FE9DF242FE7CF8B
:105D70000196272FE4DFE2CFDC01CB0102C02D9199
:105D800005D041505040D8F70895262FF999FECFFD
:105D90001FBA92BD81BD20BD0FB6F894FA9AF99A48
:105DA0000FBE01960895F894FFCF98089D089F08AC
:105DB000A408B408B408B408B408B408B408B40813
:105DC000B408A608AA08AD08B208C208C808CC08DA
:105DD000300E560E5C0E560E5C0EAE0ECF0E5C0EE6
:105DE000D50FE20FE3194B1AEB19B519B919EF19D1
:105DF000BD19F319FF19C919441ACD19031AD1197C
:105E0000071A2C1AD5190B1A331ADB19111A191A79
:105E1000C119F719C519FB19DF19151A231A3C1AEC
:105E2000421AAF19E719521A8119871974197B1987
:105E30008D1993199919AF1BAF1BE61BE61B961C16
:105E4000B11C0A1C0A1CB61C291D3A1D3A1DA72AA2
:105E5000C22AC92A03290329FC2A0D2B202B612BD6
:105E6000662B0329032903296E2BF128F5282629FF
:105E7000352940294B29EE28EE28EE28EE28922AD3
:105E80004E29512954298129BD29C029C229F62921
:0E5E9000762B842B9B2BD02BEC2B0F2C222C53
:105E9E00ED07790B8F0B940B990B700B0000010023
:105EAE000101C5647499A32A1839004422B68401ED
:105EBE006201AC008A02A302C3029694953297F750
:105ECE00F6F5F4F1F0C63031343536666793E200FC
:105EDE00E900EA00B500B600B700CD008301CC00A2
:105EEE008A01920194012102230224022502260234
:105EFE0027022A02B300B4006F0070009F01CB018D
:105F0E009F02A002E200E900EA00B500B600B70069
:105F1E00CD008301CC008A0192019401210223025B
:105F2E0024022502260227022A02B300B4006F00C3
:0A5F3E0070009F01CB019F02A0023A
:00000001FF
